:100000000AC023C022C021C020C01FC01EC01DC006
:100010001CC01BC01AC011241FBECFEDCDBF10E005
:10002000A0E6B0E0E8ECF7E003C0C89531960D9289
:10003000A037B107D1F710E0A0E7B0E001C01D92F2
:10004000A137B107E1F756D3BEC3DACFCF93DF9321
:10005000CDB7DEB7E8E3F0E01082E7E3F0E08FE051
:100060008083E2E3F0E01082E1E3F0E082E080836D
:10007000DF91CF910895CF93DF93CDB7DEB725976A
:100080000FB6F894DEBF0FBECDBF6A837B838C832F
:100090009D838A819B81AC81BD81880F991FAA1F96
:1000A000BB1F880F991FAA1FBB1F880F991FAA1F6C
:1000B000BB1F880F991FAA1FBB1F282F392F4A2F3C
:1000C0005B2F80E896E9A8E9B0E0682F792F8A2FA6
:1000D0009B2F52D3B52FA42F932F822F815089832A
:1000E000E9E2F0E089818083AAE2B0E0EAE2F0E0B0
:1000F000808188618C9325960FB6F894DEBF0FBE81
:10010000CDBFDF91CF910895CF93DF93CDB7DEB709
:1001100021970FB6F894DEBF0FBECDBF8983EBE207
:10012000F0E080819927807290700097C1F3ECE233
:10013000F0E08981808321960FB6F894DEBF0FBE70
:10014000CDBFDF91CF910895CF93DF93CDB7DEB7C9
:1001500022970FB6F894DEBF0FBECDBFEBE2F0E002
:100160008081882344F4ECE2F0E08081282F33275B
:100170003A83298302C01A82198289819A81229640
:100180000FB6F894DEBF0FBECDBFDF91CF910895BB
:10019000CF93DF93CDB7DEB723970FB6F894DEBFCA
:1001A0000FBECDBF8B831A8281E089838DE0ACDFE7
:1001B0008AE0AADF19C08B81882349F08A819927B8
:1001C000F92FE82FE05AFF4F8081898308C08A8188
:1001D0009927F92FE82FE859FF4F8081898389817A
:1001E00093DF8A818F5F8A838981882321F78DE05D
:1001F0008BDF8AE089DF23960FB6F894DEBF0FBE4F
:10020000CDBFDF91CF910895CF93DF93CDB7DEB708
:10021000A4970FB6F894DEBF0FBECDBF8A871B82AE
:1002200081E08A8380E389831C820FC08C81282F20
:1002300033278C2F9D2F0596F92FE82FE20FF31F00
:1002400080E380838C818F5F8C838C81853070F319
:100250001C828A85282F33273AA329A389A19AA132
:100260008130910509F444C029A13AA12230310519
:1002700009F4EBC026C168DF8B833B813BA38BA1D4
:10028000882311F091E09BA32BA128A31F8E8B81C3
:100290008D3011F031E03F8F88A19F8D8923282F69
:1002A00033278A81992782239323009709F11E8E91
:1002B0008B81803311F021E02E8F1D8E8B81813355
:1002C00011F031E03D8F8E8D9D8D8923882309F0BB
:1002D0001A828C81282F33278C2F9D2F0596F92F7A
:1002E000E82FE20FF31F8B8180838C818F5F8C83DB
:1002F0001C8E8B818D3011F021E02C8F1B8E8C8118
:10030000853010F431E03B8F8C8D9B8D8923282F15
:1003100033278A81992782239323009709F0ABCF53
:100320001A8E8C81853011F421E02A8F198E8A81F2
:10033000882311F431E0398F8A8D998D892B882398
:1003400019F080E025DFBDC01B821C8224C08C8197
:10035000282F33278C2F9D2F0596F92FE82FE20F9A
:10036000F31F8081482F55278C81282F332783E066
:1003700090E0821B930B242F352F02C0220F331FD6
:100380008A95E2F7932F822F982F8B81892B8B836D
:100390008C818F5F8C838C818430C8F2E8E3F0E03D
:1003A0008B8180838EC0D0DE8B833B813CA38CA16C
:1003B000882311F091E09CA32CA1288F1F8A8B81A8
:1003C0008D3011F031E03F8B888D9F898923282F54
:1003D00033278A819927822393230097B1F18C8157
:1003E0008F5F8C838B8189831E8A1D8A89818033EC
:1003F00020F421E030E03E8B2D8B1C8A89818A33EA
:1004000010F031E03C8B1B8A8981813410F481E04B
:100410008B8B8C899B89892399272D893E89282B51
:10042000392B3A8B298B188A1F868981873420F0D3
:1004300081E090E0988B8F8789899A892F85388908
:10044000822B932B009709F01A821E868B818D30A8
:1004500011F031E03E871D868C81823010F481E0FE
:100460008D878E859D858923282F33278A8199271B
:1004700082239323009709F096CF89818B831C8672
:100480008C81823011F421E02C871B868A8188239D
:1004900011F431E03B878C859B85892B882319F0EB
:1004A00080E076DE0EC08B818A3320F48B8180530E
:1004B0008B8303C08B8187538B83E8E3F0E08B81D0
:1004C0008083A4960FB6F894DEBF0FBECDBFDF9138
:1004D000CF910895CF93DF93CDB7DEB724970FB6B2
:1004E000F894DEBF0FBECDBF8A8319828A81282F80
:1004F00033273C832B838B819C818130910531F0A4
:100500002B813C8122303105B1F16DC0E0E3F0E098
:100510008081992784709070009719F481E3F4DD4D
:1005200002C080E3F1DDE0E3F0E08081992788708C
:100530009070009719F481E3E7DD02C080E3E4DD09
:10054000E0E3F0E08081992780729070009719F4C1
:1005500081E3DADD02C080E3D7DDE0E3F0E0808113
:10056000992780749070009719F481E3CDDD3BC02A
:1005700080E3CADD38C0E0E3F0E080819927847031
:100580009070009719F48981885F8983E0E3F0E037
:100590008081992788709070009719F489818C5F09
:1005A0008983E0E3F0E08081992780729070009762
:1005B00019F489818E5F8983E0E3F0E080819927D7
:1005C00080749070009719F489818F5F8983898185
:1005D0008A3020F48981805D898303C08981895CA8
:1005E0008983898191DD24960FB6F894DEBF0FBE12
:1005F000CDBFDF91CF910895CF93DF93CDB7DEB715
:100600002C970FB6F894DEBF0FBECDBF8A83198238
:100610008A81282F33273C872B878B859C858230C6
:10062000910581F0EB85FC85E330F10509F452C0BA
:100630002B853C852130310509F053C0E8E3F0E01B
:1006400010824FC0E8E3F0E08FE080834AC07CDD99
:10065000898388E390E09A878987E0E3F0E08081EE
:10066000992784709070009719F498E0988701C0DA
:100670001886E0E3F0E080819927887090700097F9
:1006800019F4E4E0EF8301C01F82F8852F81F20F97
:10069000FE83E0E3F0E080819927807290700097FC
:1006A00019F432E03D8301C01D828E819D81890F46
:1006B0008C83E0E3F0E080819927807490701B8246
:1006C000009711F4E1E0EB838C81FB818F0FE985CA
:1006D000FA8580838981833509F0B9CFE8E3F0E0BA
:1006E00010822C960FB6F894DEBF0FBECDBFDF91FF
:1006F000CF910895CF93DF93CDB7DEB7A7DC60E845
:1007000075E280E090E0B7DC00C081E041DD10924E
:10071000700003C019DD8093700080917000882301
:10072000C9F380917000873511F481E06DDD80910F
:100730007000873711F482E067DD809170008235A8
:1007400011F481E0C7DE80917000823711F482E0FD
:10075000C1DE80917000833411F481E04DDF80911F
:1007600070008F3411F482E047DF80917000833590
:1007700061F683E041DFC9CFA1E21A2EAA1BBB1BA1
:10078000EA2FFB2F0DC0AA1FBB1FEE1FFF1FA217D2
:10079000B307E407F50720F0A21BB30BE40BF50B3E
:1007A000661F771F881F991F1A9469F760957095C7
:1007B00080959095262F372F482F592F6A2F7B2F02
:0807C0008E2F9F2F0895FFCF3B
:1007C80057656C636F6D65004572726F722100002A
:00000001FF
